:1000000000308A00AD2800003C308400000803194D
:1000100018280130F800F701F70B0C28F80B0B2813
:100020004A30F700F70B122800000000800B092867
:100030008A110A12FE2883160612831206168316E8
:1000400006108312061483168610831286108316F8
:10005000061583128A110A12052983168610831247
:1000600086108316061283120612BD013D080F3C4E
:10007000031C592883168610831286100039F70056
:100080003C088039FA0077087A0403194C28831653
:1000900006108312061450288316061083120610C9
:1000A00083168610831286140310BB0DBC0DBD0A87
:1000B0003628831686108312861083160612831242
:1000C00006160034831686108312861083160612D5
:1000D000831206128316061083120610BD013D0816
:1000E0000F3C031C85288316861083128614831602
:1000F0008610831286148316861083128610831648
:10010000861083128610BD0A6F28BE01BD013D080E
:10011000073C031CA4280310BE0D8316061583128A
:1001200006193E14831686108312861483168610D1
:100130008312861483168610831286108316861007
:1001400083128610BD0A87288316061283120616AC
:100150003E08F8008A110A12462984011F308305DF
:100160001930831699002630980090308312980039
:1001700083161F149F141F159F1107309C00FF301A
:100180008312B70083161F149F141F159F1183122B
:100190001F109412B7123708831687008312371680
:1001A0003708831687008312B71137088316870034
:1001B0002030831294000030831694000108C73960
:1001C00008388100831290010030F800920000305E
:1001D0008316920007309C0005080330F700F70BE8
:1001E000EF281C0883120D1383169D0186128312BB
:1001F00086160430BB00FA30BC000428BB0BFB2879
:1002000083168612831286121B28BC01BB012D2087
:100210009130BC008A30BB002D20A630BC0040309D
:10022000BB002D20C830BC004730BB002D20C6309D
:10023000BC009B30BB002D20C430BC002A30BB006A
:100240002D20C230BC004030BB002D20C030BC008F
:100250008030BB002D20CE30BC008830BB002D206C
:10026000CE30BC008B30BB002D20C030BC008130B4
:10027000BB002D203610B80183168615831286190F
:100280007F293808B80A203EBC0062283C08840058
:100290007808800001303802203E84000008BC004D
:1002A0003C080C1E512999003808123C031D7E2978
:1002B000B801CE30BC008830BB002D20CE30BC0051
:1002C0008B30BB002D20BA01B90139080F3C031C4B
:1002D00070292030390784000008BA07B90A652957
:1002E00030083A02031D7E290130B60636187A29F5
:1002F00086127B2986168316861283123C293C2996
:02030000630098
:02400E00393F38
:00000001FF
